:020000040000FA
:10000000F2EF03F01200FFFF04EF04F01200FFFF15
:10001000FFFFFFFFFFFFFFFF0CEF04F012000000E7
:100020000001776B1E0E716E0401400E096F200EE9
:100030000A6F040E0B6F880E086F0401200E0E6FFE
:10004000040E0F6F400E0C6F1200550EA76EAA0E15
:10005000A76EA68212000401226B010E236F12000C
:100060000001756B040121510001755D20E275C02E
:1000700000F0016A026A040122510024F36E235148
:100080000120F46E24510220F86EF4CFF7FFF3CF75
:10009000F6FF0800F5CF76F000017551EA6A250FEA
:1000A000E96E040EEA2276C0EFFF752BDBD7F86A03
:1000B0001200F00E04012217840EA66E0001756B6B
:1000C000040121510001755D26E27551EA6A250F90
:1000D000E96E040EEA22EFCF03F075C000F0016A6A
:1000E000026A040122510024F36E23510120F46EB0
:1000F00024510220F86EF4CFF7FFF3CFF6FF03C0D0
:10010000F5FF0C000F0E000175150F0801E19DDFD2
:100110000001752BD5D71200940EA66E0001756BE9
:10012000040121510001755D1EE27551006E016AE6
:10013000060ED89000360136E804FBE1026A01BEE3
:100140000268040122510024F36E23510120F46E51
:1001500024510220F86EF4CFF7FFF3CFF6FF75DFDE
:100160000001752BDDD7F86A1200A66A0001756BD5
:10017000040121510001755D10E2040122510001CA
:100180007525A96EA6807551EA6A250FE96E040EE1
:10019000EA22A8CFEFFF752BEBD712000001756B99
:1001A000040121510001755D15E204012251000195
:1001B0007525A96E7551EA6A250FE96E040EEA22CB
:1001C000EF50A86E040EA66E40DFA6B2FED7000167
:1001D000752BE6D71200C40EA66E0001756B0401E4
:1001E00021510001755D21E27551EA6A250FE96E22
:1001F000040EEA22EFCF03F075C000F0016A026A34
:10020000040122510024F36E23510120F46E245185
:100210000220F86EF4CFF7FFF3CFF6FF03C0F5FF2F
:100220000C0013DF0001752BDAD7F86A12008BD8A7
:10023000060E00017C5D03E36D50020B01E082D0ED
:100240000001770511E104010CBF0DD00401400E3F
:10025000096F400E040108170401087D880E04018F
:1002600008130001776B6ED0040108BF6BD000014A
:10027000756B04012051320A45E0CD0A34E0F80ADA
:100280002DE0020A26E0010A1FE0070A18E0010A31
:1002900011E0030A0AE0070A08E0060A01E041D07B
:1002A000DADE0001040E756F3DD0DADE050E0001C6
:1002B000752738D0FEDE0001010E756F33D02CDFBC
:1002C0000001010E756F2ED050DF050E000175275D
:1002D00029D064DF0001010E756F24D07CDF00019E
:1002E000010E756F1FD06D960001786B796B000160
:1002F0007807000E795B00017851791101E0F7D79A
:10030000FF0010D0030E0401215D03E10001010E86
:10031000756F040E0401215D03E10001010E756F8C
:1003200001D000D00001010E776F000175510AE085
:1003300075C00DF4400E04010C1704010C7D880EED
:1003400004010C131200060E00017C5D10E1000197
:100350007A517B1105E18B82200E7A6F4E0E7B6FF6
:10036000880E7A1904E1130E7B1901E18B920001CA
:100370007A07000E7B5B12006C5002E0000E01D089
:10038000010E00090BE0040100513C0BE842E84279
:100390000D0802E1D7EF01F0E0EF01F06C5002E050
:1003A000000E01D0010E040901E019D8120000016D
:1003B000606B616B666B676BB5EC02F062EF02F02D
:1003C000020E0001605D09E15CD8040100BD02D0AD
:1003D000C80E01D0880E006F1200A7EF02F0040EC5
:1003E00000017C5D09E112C46EFF6E50000802E25C
:1003F000050E01D0030E7C6F0001600509E10AD8EB
:10040000040104BD02D0C80E01D0880E046F120092
:10041000A7EF02F00001080E665D000E675903E2C7
:1004200066C069F002D0080E696F69C005F46951B1
:10043000006E016A0050665F0150675B180E646FC2
:10044000040E656F69511CE000017DA307D062C0F6
:10045000F6FF63C0F7FF0800F55005D062C0E9FF62
:1004600063C0EAFFEF5064C0E9FF65C0EAFFEF6ECA
:100470000001622B000E6323642B65236907E2D71A
:10048000120001C46AF000016A516625666F000E11
:100490006721676F180E626F040E636F6A5111E077
:1004A00062C0E9FF63C0EAFFEF5064C0E9FF65C0C6
:1004B000EAFFEF6E642B000E6523622B63236A074D
:1004C000EDD71200000161510BE10401080E016F2C
:1004D000100E026F040E036F840E006F040123D010
:1004E000040110AF22D0000166510401165D000125
:1004F00067510401175904E216C466F017C467F087
:1005000089DF0001010E606F0401080E016F100EFB
:10051000026F040E036F800E006F0401180E066F49
:10052000040E076FC80E046F10D00001020E606F3A
:100530000401056BC80E046F0401080E016F180E4C
:10054000026F040E036FC80E006F6D981200000159
:10055000606B0401080E016F100E026F040E036F32
:10056000880E006F0401046B120004011051600B2F
:10057000E842E842E842E842E842000901E01200AD
:100580001151080A39E0010A35E00F0A0AE0030AAE
:1005900001E012000001010E616F0001040E7C6F8A
:1005A00012000001010E616F0401130507E1000153
:1005B0007E0E626F070E636F120E13D0020E135D74
:1005C00007E10001900E626F070E636F200E09D0E5
:1005D000030E135D0AE10001B00E626F070E636F38
:1005E000040E0001666F676B02D00001616B0001B1
:1005F0007D8312000AEF03F00001010E616F00011C
:100600007E0E626F000E636F00017D930001010E8C
:10061000666F12000001010E616F12C47EF00401CA
:10062000125104E10001050E7C6F12000001060E5C
:100630007C6F10EF00F0080E6D6E6DBAFED7686A21
:10064000110E696E0001020E7C6F12006850040BDF
:1006500006E06950040B03E06D9269946894685059
:10066000010B04E06950010B01E027D86850100B22
:1006700009E06950100B06E0698468986D82A08AD1
:100680000300A19A6850200B09E06950200B06E096
:1006900070A003D0A7EC02F07090689A030E0001DE
:1006A0007C5D01E209D06850080B06E06950080B38
:1006B00003E0BCEC01F068961200686A7B0E696E7C
:1006C0006E6A160E706E68A602D06896FCD76D989A
:1006D000A7EC02F000017E6B0001030E7C6F12009C
:1006E0001E0EF66E000EF76E000EF86E0001090089
:1006F000F550706F0900F550716F03E1706701D01C
:100700003DD00900F5506B6F0900F5506C6F090082
:10071000F5506D6F09000900F550E96E0900F550BC
:10072000EA6E090009000900F5506E6F0900F550E6
:100730006F6F09000900F6CF72F0F7CF73F0F8CFB2
:1007400074F06BC0F6FF6CC0F7FF6DC0F8FF0001DE
:100750006E5302E16F5307E00900F550EE6E6E072D
:10076000F8E26F07F9D772C0F6FF73C0F7FF74C0E5
:10077000F8FF00017007000E715BBFD71200120175
:10078000000200000008D8040B0000000000000177
:10079000090220000101008032090400000200006B
:1007A000000007050102400000070581024000002B
:1007B00004030904C1CF80F00F0EC11282A404D03B
:1007C00080C0C1FF00EF04F0FC0E8B16FC0E9416E7
:1007D000140E6F6E1BEC03F026EC03F017EC01F027
:1007E000FBD7120013EE00F023EE00F0F86A059C30
:1007F00070EC03F0DAEC03F0FDD71200FFFFFFFF0F
:10080000FFFFFFFFFFFFFFFFFFFFFFFFFFFFFFFFF8
:10081000FFFFFFFFFFFFFFFFFFFFFFFFFFFFFFFFE8
:10082000FFFFFFFFFFFFFFFFFFFFFFFFFFFFFFFFD8
:10083000FFFFFFFFFFFFFFFFFFFFFFFFFFFFFFFFC8
:0200000400F00A
:020000040030CA
:0E0000002002321EFF8081FFFFFFFFBFFFFFC7
:020000040020DA
:08000000FFFFFFFFFFFFFFFF00
:00000001FF
